:020000040800F2
:100000000000022019120008B9110008BB110008F5
:10001000BD110008BF110008C11100080000000058
:10002000000000000000000000000000C3110008F4
:10003000C511000800000000C7110008C911000820
:1000400069120008691200086912000869120008A4
:100050006912000869120008691200086912000894
:100060006912000869120008691200086912000884
:100070006912000869120008691200086912000874
:1000800069120008691200086912000800000000E7
:1000900000000000000000000000000069120008DD
:1000A0006912000869120008691200086912000844
:1000B0006912000869120008691200086912000834
:1000C0006912000869120008691200086912000824
:1000D0006912000869120008691200080000000097
:1000E0006912000869120008691200080000000087
:1000F000000000000000000000000000691200087D
:100100000000000069120008691200086912000866
:1001100000000000000000000000000000000000DF
:1001200069120008691200086912000869120008C3
:10013000691200080000000000000000000000003C
:10014000000000000000000000000000691200082C
:100150006912000869120008691200086912000893
:100160006912000869120008000000000000000089
:10017000000000000000000000000000000000007F
:1001800000000000691200080000000000000000EC
:08019000691200086912000861
:1001980010B5054C237833B9044B13B10448AFF3B9
:1001A80000800123237010BD0C0000200000000017
:1001B800C412000808B5034B1BB103490348AFF349
:1001C800008008BD0000000010000020C4120008D4
:1001D80053B94AB9002908BF00281CBF4FF0FF31A6
:1001E8004FF0FF3000F07AB9ADF1080C6DE904CE9C
:1001F80000F006F8DDF804E0DDE9022304B07047FA
:100208002DE9F0478C460D460446089E002B51D137
:100218008A4217466DD9B2FA82FEBEF1000F0BD0A2
:10022800CEF1200C01FA0EF520FA0CFC02FA0EF7BA
:100238004CEA050C00FA0EF44FEA174A250CBCFBF1
:10024800FAF81FFA87F90AFB18CC45EA0C4508FBAF
:1002580009F3AB420AD9ED1908F1FF3280F0238186
:10026800AB4240F22081A8F102083D44ED1AA4B245
:10027800B5FBFAF00AFB105544EA054400FB09F9FE
:10028800A14509D9E41900F1FF3380F00A81A1459D
:1002980040F2078102383C44A4EB090440EA0840D4
:1002A8000021002E61D024FA0EF40023346073601C
:1002B800BDE8F0878B4207D9002E54D0002186E88C
:1002C80021000846BDE8F087B3FA83F1002940F021
:1002D8008E80AB4202D3824200F2FA80841A65EB28
:1002E80003050120AC46002E3FD086E81010BDE87B
:1002F800F08712B90127B7FBF2F7B7FA87FEBEF10C
:10030800000F34D1EB1B3A0C1FFA87FC0121B3FB19
:10031800F2F8250C02FB183345EA03450CFB08F3F9
:10032800AB4207D9ED1908F1FF3002D2AB4200F217
:10033800D1808046ED1AA3B2B5FBF2F002FB10554E
:1003480043EA05440CFB00FCA44507D9E41900F175
:10035800FF3302D2A44500F2B8801846A4EB0C047F
:1003680040EA08409DE731463046BDE8F087CEF1C7
:10037800200405FA0EF307FA0EF720FA04F83A0CEF
:1003880025FA04F448EA0308B4FBF2F14FEA1845E9
:1003980002FB11441FFA87FC45EA044501FB0CF3F4
:1003A800AB4200FA0EF409D9ED1901F1FF3080F0E3
:1003B8008A80AB4240F2878002393D44EB1A1FFA2B
:1003C80088F5B3FBF2F002FB103345EA034500FB66
:1003D8000CF3AB4207D9ED1900F1FF386FD2AB42ED
:1003E8006DD902383D44EB1A40EA01418FE7C1F16B
:1003F800200722FA07F88B4005FA01F448EA0303BC
:1004080020FA07FE4FEA134CFD404EEA040EB5FBF6
:10041800FCF94FEA1E440CFB19551FFA83F844EA0D
:10042800054509FB08F4AC4202FA01F200FA01FAA8
:1004380008D9ED1809F1FF3043D2AC4241D9A9F1EE
:1004480002091D442D1B1FFA8EFEB5FBFCF00CFBA8
:1004580010554EEA054400FB08F8A04507D9E418F2
:1004680000F1FF3529D2A04527D902381C4440EABB
:100478000940A4EB0804A0FB02894C45C6464D463A
:1004880015D312D056B1BAEB0E0364EB050404FA87
:1004980007F7CB401F43CC40376074600021BDE8AC
:1004A800F0871846F8E69046E0E6C245EAD2B8EB8F
:1004B800020E69EB03050138E4E72846D7E7404612
:1004C80091E78146BEE7014678E702383C4445E7B4
:1004D800084608E7A8F102083D442BE7704700BF2B
:1004E80038B50E4A0E4B054618784FF47A73B3FBAD
:1004F800F0F31068B0FBF3F000F09CF8044658B92C
:100508000F2D09D8024629464FF0FF3000F05EF85B
:10051800044B20461D6038BD012038BD080000206E
:10052800000000200400002008B50B4B1A6842F4B4
:1005380000721A601A6842F480621A601A6842F4FB
:1005480080721A60032000F02FF80020FFF7C8FF20
:1005580000F0D6FD002008BD003C0240034A044BD1
:1005680011681B780B441360704700BF28000020F7
:1005780000000020014B1868704700BF28000020C9
:1005880038B50446FFF7F6FF631C1CBF054B1B7804
:10059800054618BFE418FFF7EDFF401B8442FAD860
:1005A80038BD00BF00000020074AD36823F4E06389
:1005B8001B041B0C43F0BF63000243F4003300F438
:1005C800E0600343D360704700ED00E0174B30B59F
:1005D800DC68C4F30224C4F10703251D042B28BFDB
:1005E8000423062D4FF0010505FA03F303F1FF3349
:1005F8008CBF033C00241940A14005FA04F4013CD7
:100608002240002842EA01024FEA0212ADBF00F17F
:10061800604000F00F00064B00F56140B5BFD2B254
:10062800D2B21A5480F8002330BD00BF00ED00E0BC
:1006380014ED00E00138B0F1807F0AD2064B074A7A
:100648005860F02182F823100020072298601A6071
:1006580070470120704700BF10E000E000ED00E0A7
:100668002DE9F04F85B00B68DFF89C81644A01934F
:100678004FF001090023019C09FA03F707EA040671
:10068800B74240F0AD804C6824F0100ABAF1020F6E
:1006980016D14FEAD30C00EB8C0C03F0070BDCF8F7
:1006A80020504FEA8B0B4FF00F0E0EFA0BFE25EA87
:1006B8000E0E0D6905FA0BF545EA0E05CCF820502B
:1006C8004FEA430C0325D0F800B005FA0CF5ED43CA
:1006D80004F0030E0BEA050B0EFA0CFE0AF1FF3AC2
:1006E8004EEA0B0EBAF1010F0095C0F800E015D8DC
:1006F800D0F808E005EA0E0ECD6805FA0CFA4AEAC9
:100708000E0EC0F808E0D0F804E02EEA0707C4F39C
:10071800001E0EFA03FE4EEA07074760C768009DF1
:100728003D408F6807FA0CF73D43C560E50057D593
:100738004FF0000BCDF80CB0D8F84470314D47F4A9
:100748008047C8F84470D8F8447007F48047039786
:10075800039F23F0030707F1804707F59C3703F051
:10076800030CD7F808A04FEA8C0C4FF00F0E0EFAC6
:100778000CFEA8422AEA0E0E39D005F58065A8427B
:1007880037D005F58065A84235D005F58065A842C3
:1007980033D005F58065A84214BF0725042505FA5E
:1007A8000CF545EA0E05BD601568F74314F4803F63
:1007B8000CBF3D4035431560556814F4003F0CBF2D
:1007C8003D4035435560956814F4801F0CBF3D408B
:1007D80035439560D568A40254BF3D403543D56084
:1007E8000133102B7FF447AF05B0BDE8F08F5D46AD
:1007F800D5E70125D3E70225D1E70325CFE700BFD9
:10080800003C014000000240003802400AB181610A
:1008180070470904FBE7436931EA030308BF090489
:10082800816170472DE9F341044618B9012002B0EF
:10083800BDE8F0810368DD0710D42368980758D411
:1008480023681A0700F19A8023685B0700F1B880D3
:10085800A269002A40F019810020E8E7A64B9A68AF
:1008680002F00C02042A07D09A6802F00C02082A47
:100878000AD15B68590207D59F4B1B689A03DCD5E0
:100888006368002BD9D1D1E763689B4DB3F5803FEE
:1008980011D12B6843F480332B60FFF76BFE964D24
:1008A80006462B689B03C8D4FFF764FE801B6428A8
:1008B800F7D90320BBE7B3F5A02F04D12B6843F485
:1008C80080232B60E5E72A6822F480322A602A68B0
:1008D80022F480222A60002BDFD1FFF74BFE064668
:1008E8002B689F03A9D5FFF745FE801B6428F7D91D
:1008F800DFE7814B9A6812F00C0F07D09A6802F074
:100908000C02082A11D15B685E020ED47A4B1A6871
:10091800950702D5E268012A88D11A68216922F070
:10092800F80242EAC1021A608AE7E268734BB2B180
:1009380001221A60FFF71EFE6F4D06462B689807C6
:1009480007D52B68226923F0F80343EAC2032B601A
:1009580076E7FFF70FFE801B0228EFD9A9E71A6098
:10096800FFF708FE644D06462B6899077FF568AFC8
:10097800FFF700FE801B0228F6D99AE76269604BF0
:100988007AB101221A60FFF7F5FD5B4D06466B6FE1
:100998009F073FF559AFFFF7EDFD801B0228F6D9F9
:1009A80087E71A60FFF7E6FD534D06466B6F980719
:1009B8007FF54AAFFFF7DEFD801B0228F6D978E7FE
:1009C8004D4B1A6C12F0805228D101921A6C42F0E9
:1009D80080521A641B6C03F080530193019B01261B
:1009E800484D2B68D9051BD5A368434D012B27D14A
:1009F8002B6F43F001032B67FFF7BCFD3E4D074605
:100A080041F288382B6F9B0739D5002E3FF420AF71
:100A1800394A136C23F08053136419E70026DFE783
:100A28002B6843F480732B60FFF7A4FD07462B68FF
:100A3800DA05D9D4FFF79EFDC01B0228F7D938E79D
:100A4800052B04D12B6F43F004032B67D0E72A6FE3
:100A580022F001022A672A6F22F004022A67002B7B
:100A6800CAD1FFF787FD41F2883807462B6F9807F0
:100A7800CBD5FFF77FFDC01B4045F7D919E7FFF736
:100A880079FDC01B4045BDD913E71B4DAB6803F08A
:100A98000C03082B3FF4CAAE1B4E0023022A336016
:100AA80034D1FFF767FD07462B6899011ED4226AE7
:100AB800E3691343626A43EA8213E26A43EA026320
:100AC800A26A0D4C5208013A43EA02436B600123C3
:100AD8003360FFF74FFD054623689A013FF5BCAE2A
:100AE800FFF748FD401B0228F6D9E2E6FFF742FD72
:100AF800C01B0228D8D9DCE6003802400000474273
:100B0800800E47420070004060004742FFF732FD08
:100B180004462B689B017FF59FAEFFF72BFD001B5A
:100B28000228F6D9C5E600BF134908B58B6803F05B
:100B38000C03042B03D0082B03D0104808BD104821
:100B480008BD4A684B68496813F4800314BF0C4811
:100B58000A48C1F3881118BF002302F03F02A1FB25
:100B68000001FFF735FB044B5B68C3F30143013316
:100B78005B00B0FBF3F008BD003802400024F4002D
:100B880000127A002DE9F0410D46044610B9012003
:100B9800BDE8F081444B1A6802F00F028A4228D35C
:100BA80021688F072DD4C80740D43F4B1A6802F03C
:100BB8000F02954266D3226851076CD4130707D5F4
:100BC8003A4A2169936823F4604343EAC103936076
:100BD800FFF7AAFF354B364A9B68C3F30313D35C70
:100BE800D840344B18600020FFF77AFC0020BDE89D
:100BF800F081CAB21A701B6803F00F039942C6D17C
:100C0800CEE72A4B11F0040F1EBF9A6842F4E05257
:100C18009A600E0742BF9A6842F460429A609A68E6
:100C2800A06822F0F00202439A60BCE762681F4B9A
:100C3800012A1DD11B6813F4003FA8D01B4EB368CE
:100C480023F003031343B360FFF794FC41F28838A1
:100C58000746B368626803F00C03B3EB820FA4D0B5
:100C6800FFF788FCC01B4045F3D90320BDE8F0819D
:100C7800911E01291B6802D813F0007FDDE713F0ED
:100C8800020FDAE7EAB21A701B6803F00F039D42FD
:100C98007FF47DAF8FE70549E0688B6823F4E05364
:100CA80003438B608AE700BF003C024000380240E3
:100CB800DC12000808000020044B054A9B68C3F3B7
:100CC8008223D35C034A1068D8407047003802403A
:100CD800EC12000808000020044B054A9B68C3F387
:100CE8004233D35C034A1068D8407047003802404A
:100CF800EC120008080000202DE9F0470668C268D9
:100D08003369C16923F4405313433361044683684C
:100D18000069F2680343606922F41642034322F033
:100D28000C020B431343F3607369A26923F4407305
:100D38001343B1F5004F73617A4B7CD19E4203D0C7
:100D480003F580639E4244D1FFF7C6FF192505FBD2
:100D580000F360684FF064094000B3FBF0F3B3FBA5
:100D6800F9F34FEA0318FFF7B7FF636868435B00BE
:100D7800B0FBF3F7FFF7B0FF636868435B00B0FBB5
:100D8800F3F3B3FBF9F309FB1373DB003233B3FB63
:100D9800F9F35B0003F4F877FFF79EFF6268684396
:100DA8005200B0FBF2FAFFF797FF636868435B00F5
:100DB800B0FBF3F3B3FBF9F309FB13A3DB00323306
:100DC800B3FBF9F303F0070343443B44B360BDE8C6
:100DD800F087FFF771FF192505FB00F360684FF0F6
:100DE80064094000B3FBF0F3B3FBF9F34FEA0318CF
:100DF800FFF762FF636868435B00B0FBF3F7FFF738
:100E08005BFF636868435B00B0FBF3F3B3FBF9F384
:100E180009FB1373DB003233B3FBF9F35B0003F414
:100E2800F877FFF749FF626868435200B0FBF2FAAF
:100E3800FFF742FFB9E79E4202D03B4B9E4240D1AA
:100E4800FFF74AFF676819254FF0640905FB00F3AF
:100E5800BF00B3FBF7F3B3FBF9F31F01FFF73CFF48
:100E6800636868439B00B0FBF3F8FFF735FF6368DE
:100E780068439B00B0FBF3F3B3FBF9F309FB13835F
:100E88001B013233B3FBF9F303F0F008FFF724FF3B
:100E9800626868439200B0FBF2FAFFF71DFF6368CF
:100EA80068439B00B0FBF3F3B3FBF9F309FB13A30F
:100EB8001B013233B3FBF9F303F00F0343EA0803D2
:100EC80083E7FFF7F9FE676819254FF0640905FB0A
:100ED80000F3BF00B3FBF7F3B3FBF9F31F01FFF710
:100EE800EBFE636868439B00B0FBF3F8FFF7E4FE92
:100EF800636868439B00B0FBF3F3B3FBF9F309FBAA
:100F080013831B013233B3FBF9F303F0F008FFF747
:100F1800D3FE626868439200B0FBF2FAFFF7CCFE9A
:100F2800BDE700BF001001400014014010B50446A1
:100F380040B390F8393003F0FF021BB980F838202D
:100F480000F0FEF82268242384F83930D36823F4AB
:100F58000053D3602046FFF7CFFE23681A6922F4B6
:100F680090421A615A6922F02A025A61DA6842F4F8
:100F78000052DA6000202023E06384F8393084F8D6
:100F88003A3010BD012010BD30B595B03022002197
:100F980008A800F08BF90021142203A800F086F9B4
:100FA80000241B4B01941A6C42F080521A641B6C8B
:100FB80003F080530193019B164B02941A6842F484
:100FC80040421A601B680F9403F440430293029B4B
:100FD80001230B9310230C930823109364230225F9
:100FE800119308A80423139308950E951295FFF7FB
:100FF80019FC0F23039303214FF4805303A804958E
:10100800059406930794FFF7BDFD15B030BD00BFEA
:10101800003802400070004000B58BB0FFF784FA3A
:10102800FFF7B2FF142200210DEB020000F03EF999
:1010380000242D4B01941A6B2C4842F004021A63C9
:101048001A6B02F004020192019A02941A6B42F0A0
:1010580080021A631A6B02F080020292029A0394C9
:101068001A6B42F001021A631A6B02F00102039232
:10107800039A04941A6B42F002021A631B6B03F082
:101088000203224604932021049BFFF7BFFB4FF481
:101098000053059305A9164B164806930794FFF7C6
:1010A800DFFA2023059305A9012310480693079426
:1010B8000894FFF7D5FA1048104A84604FF4E133DA
:1010C80080E80C000C23C46004618461C46143613E
:1010D800FFF72CFF054C20462021FFF79CFBC8207A
:1010E800FFF74EFAF7E700BF003802400000024061
:1010F80000002110000802402C000020004400409D
:1011080007B50E4B002100915A6C42F480425A6494
:101118005A6C02F480420092009A01911A6C42F0D3
:1011280080521A641B6C03F0805301930720019BC3
:10113800FFF73AFA03B05DF804FB00BF003802403D
:1011480010B5044688B01422002103A800F0AEF8B8
:101158002268154B9A4224D103F5FA3300210191F4
:101168001A6C124842F400321A641A6C02F4003203
:101178000192019A02911A6B42F001021A631B6BE9
:1011880003F001030293029B0C23039302230493AD
:10119800012305930323069303A907230793FFF766
:1011A8005FFA08B010BD00BF0044004000000240D4
:1011B8007047FEE7FEE7FEE7FEE7704770477047B7
:1011C800FFF7CCB90F49D1F8883043F47003C1F860
:1011D80088300D4B1A68002042F001021A609860AE
:1011E8001A6822F0847222F480321A60074A5A6020
:1011F8001A6822F480221A60D8604FF000638B606E
:10120800704700BF00ED00E00038024010300024B5
:10121800DFF834D0002103E00C4B5B584350043115
:101228000B480C4B42189A42F6D30B4A02E00023B3
:1012380042F8043B094B9A42F9D3FFF7C3FF00F089
:1012480011F8FFF7E9FE70470000022004130008B8
:10125800000000200C0000200C0000206C00002082
:10126800FEE7000070B50D4E0D4CA41BA410002520
:10127800A54209D10B4E0C4C00F020F8A41BA41079
:101288000025A54205D170BD56F82530984701358F
:10129800EEE756F8253098470135F2E7FC120008CA
:1012A800FC120008FC120008001300080244034660
:1012B800934200D1704703F8011BF9E7F8B500BF66
:1012C800F8BC08BC9E467047F8B500BFF8BC08BC1F
:0412D8009E46704777
:1012DC0000000000000000000102030406070809DA
:0812EC000000000001020304F0
:0812F40014EFFF7F0100000070
:0412FC00BD01000828
:041300009901000847
:0C13040001000000100000000024F400B4
:0400000508001219C4
:00000001FF
